:020000040800F2
:10000000600600206D0100087101000873010008FE
:100010007501000877010008790100080000000060
:100020000000000000000000000000007B0100084C
:100030007D010008000000007F0100088101000828
:100040008301000883010008830100088301000880
:100050008301000883010008830100088301000870
:100060008301000883010008830100088301000860
:100070008301000883010008830100088301000850
:100080008301000883010008830100088301000840
:100090008301000883010008830100088301000830
:1000A0008301000883010008830100088301000820
:1000B0008301000883010008830100088301000810
:1000C0008301000883010008830100088301000800
:1000D00083010008830100088301000883010008F0
:1000E00083010008830100088301000800F002F882
:1000F00000F02CF80AA090E8000C82448344AAF196
:100100000107DA4501D100F021F8AFF2090EBAE893
:100110000F0013F0010F18BFFB1A43F0010318473B
:100120006003000070030000002300240025002667
:10013000103A28BF78C1FBD8520728BF30C148BF4A
:100140000B6070471FB51FBD10B510BD00F02DF836
:100150001146FFF7F7FF00F03FF900F04BF803B44A
:10016000FFF7F2FF03BC00F053F800000848804797
:10017000FEE7FEE7FEE7FEE7FEE7FEE7FEE7FEE757
:10018000FEE7FEE703480449044A054B70470000B8
:10019000ED000008600000206006002060020020E2
:1001A00060020020704770477047754600F02CF8D9
:1001B000AE4605006946534620F00700854618B054
:1001C00020B5FFF7DFFFBDE820404FF000064FF0FD
:1001D00000074FF000084FF0000B21F00701AC467C
:1001E000ACE8C009ACE8C009ACE8C009ACE8C0099B
:1001F0008D46704710B50446AFF300802046BDE839
:100200001040FFF7ACBF000000487047000000201E
:1002100001491820ABBEFEE726000200704700B57A
:100220000021012000F08AF80021022000F086F869
:1002300000BD70B505460E460DB9002400E040240F
:10024000344344F08000002100F078F870BD0000D5
:1002500000B51F48806940F00C001D4988611D48A9
:100260001D4908604FF044301C4908601A480C30A2
:10027000006820F0F30018490C3108604FF4FA4090
:1002800000F09EF84FF4FA4000F09AF84FF4FA406C
:1002900000F096F810480C30006820F001000E497C
:1002A0000C3108600846006820F002000860202039
:1002B000086000F023F80021282000F03FF800211A
:1002C0000E2000F03BF80021062000F037F800BDBA
:1002D0000010024033003333000C0140000801409D
:1002E00030B505462C4604E02078012100F026F8C0
:1002F000641C14B120780028F6D130BD00B50E483A
:10030000006820F002000C490860DC2000F058F87A
:100310000948006840F0020007490860DC2000F04E
:100320004FF80548006820F0020003490860DC200F
:1003300000F046F800BD00000C0C014030B504464A
:100340000D461E48006820F0F3001C49086008466E
:10035000006804F0F001084318490860012D05D138
:100360000846006840F00100086005E01348006896
:1003700020F0010011490860FFF7C0FF0F48006836
:1003800020F0F3000D4908600846006804F00F01F2
:1003900040EA011009490860012D05D108460068AE
:1003A00040F00100086005E00448006820F001000A
:1003B00002490860FFF7A2FF30BD00000C0C0140AD
:1003C0000022002104E000E0521C3C2AFCDB491C16
:1003D0008142F8DB70470000FFF73AFFFFF71FFF8D
:1003E00002210020FFF725FF19A0FFF779FF09215F
:1003F0000120FFF71EFF1AA0FFF772FF26E002217F
:100400000020FFF716FF12A0FFF76AFF4FF47A7083
:10041000FFF7D6FF1348006800F0010058B1012132
:100420000846FFF706FF10A0FFF75AFF40F2DC5026
:10043000FFF7C6FF0AE001210846FFF7FAFE0DA00C
:10044000FFF74EFF40F2DC50FFF7BAFFD7E700009E
:10045000456D6265646465642047726F7570000065
:100460004F37000008080140427574746F6E204FCA
:100470006E200000427574746F6E204F6666000037
:100480009004000800000020600600002801000819
:04000005080000ED02
:00000001FF
